:030000000239E0E2
:0C39E00078FFE4F6D8FD758155023A2707
:102445000A53746172743A20004950436F6E6E6589
:1024550063745245510A00444843502D4F4B0A00BE
:102465004950436F6E6E65637400C0E4E0EFF2E5BA
:10247500F020D1E8EDEAEEEC4950284343290A0063
:10248500C2E5F0F1E8FF20495020ECEEE4F3EBFF64
:102495003A20322E3420EEF22032302E31312E32D7
:1024A5003030350A00C4E0F2E020F1EEE7E4E0ED7B
:1024B500E8FF3A200053657020323620323030363E
:1024C50000200031313A32313A3337000A000A50E0
:1024D500524F473A20202020202020202020202055
:1024E50020202020202020202020202020202020E7
:1024F50020202020202020202020202020202020D7
:1025050020202020202020202020202020202020C6
:102515002020202020202020200A0044756D70589E
:102525002020202020303020303120303220303320
:1025350020303420303520303620303720303820D8
:102545003039203041203042203043203044203083
:10255500452030460A003A200044756D704420201D
:1025650020202030302030312030322030332030D0
:10257500342030352030362030372030382030397F
:102585002030412030422030432030442030452047
:1025950030460A00457272206B65790052642065E9
:1025A5006570726F6D0A005264204D454D0A0044F6
:1025B500656275674950204F4E0A0044656275672C
:1025C5004950204F46460A00446562756755736554
:1025D50072204F6E0A0044656275675573657220F7
:1025E5004F46460A0044656275674D7367204F6E16
:1025F5000A0044656275674D7367204F46460A00B9
:10260500436F6E666967206C6F636B210A005772B2
:1026150020656570726F6D0A0020536176652065CF
:102625006570726F6D210A00457272204D4143211C
:10263500004C6F61643E3E00576169745265737466
:1026450061727421004E4F4950004C494E4B434F27
:102655004E5452005452415353004652004E4F4C73
:10266500494E4B00494E490000FF264AFF264FFFC1
:0E2675002659FF265FFF2662FF2669FF266DAD
:06423600015200015000DE
:1041CC00C2AFC28E758900438910758BFF758DB790
:0741DC00D2ABD28ED2AF225C
:03001B0002394A5D
:10394A00C0E0C083C082C0D0C2AFC28E758BFF7583
:10395A008DB720190675A61E75A6E10550D215E584
:10396A0052600205520555E555540F7053D220E5B1
:10397A0055543F7014D213906E48E0600C04F0E086
:10398A00D394B44004C2AF80FE906E43E060020458
:10399A00F0E551D3940140021551906940E060026C
:1039AA0014F0906E49E0D394014003E014F030180B
:1039BA00020553E554D394644004D2198002055495
:1039CA00E54FD394014002154FD28ED2AFD0D0D05A
:0639DA0082D083D0E03230
:10405100E4FFFEFD74162DF582E4346BF583E02F49
:10406100FFE43EFE0DBD10ECE4FD746B2DF582E422
:104071003469F583E0FC2FFFE43EFEEC60040DBDE6
:0240810080E8D5
:01408300221A
:100A1A00C291C290C21D7D027C007F071241798F6C
:100A2A003CE53C646060097D017F60124114D21D7F
:100A3A00E4FDFC7F0B1241798F3CE53C30E6097DF1
:100A4A0004E4FF124138D21D7D017C007F07124168
:100A5A00798F3CE53C7008FD7FFF124114D21D30AE
:100A6A001D03126000C2AFC288D2A8C2AA123C7685
:100A7A00C291D290D2AF124051122889D291C2901B
:100A8A00906E441220B600000000E47F207E4EFDE6
:100A9A00FC906E44E0F8A3E0F9A3E0FAA3E0FBC3FC
:100AAA001220835027906E44E0FCA3E0FDA3E0FEF1
:100ABA00A3E0FFE4FAF9F8EF2401FFEA3EFEE93D7C
:100ACA00FDE83CFC906E441220AA80BED291D290DE
:100ADA001232F1C219C291D290123ED7D291C2906B
:100AEA00906B14E0C3940350037403F0D21FD21E18
:100AFA00D21DD293201D077E247F451233E2E49053
:100B0A006D34F01241CCC2AF755101A3F0C21AC2C2
:100B1A001BD2AF75A70775A61E75A6E1124196D21C
:100B2A0091D290906E441220B600000000E47F201B
:100B3A007E4EFDFC906E44E0F8A3E0F9A3E0FAA330
:100B4A00E0FBC31220835027906E44E0FCA3E0FD33
:100B5A00A3E0FEA3E0FFE4FAF9F8EF2401FFEA3E7E
:100B6A00FEE93DFDE83CFC906E441220AA80BEC21C
:100B7A0091C290201D19AF3C7E007D031234C7E458
:100B8A00FF1237FA7E6B7F34E4FB7D011235A590A4
:100B9A006E48E060037401F0E4906940F0A3745574
:100BAA00F0A37481F0E4F553E4F554906940E070E1
:100BBA0003122683906E49E0B401119080007410EC
:100BCA00F0E4906E49F0D21DD21ED21FE553D394A1
:100BDA0003402D908002E4F0908001F0908000F0B4
:100BEA00E553D3940540037401F0E553D3940A40C6
:100BFA000FE4F553C216906D35F0755101123ED7C8
:100C0A009080A0E070077FCB7E03123B769080B87D
:100C1A00E070031238A89080D0E07014302111904F
:100C2A006E3F74FFF0906B08E0FEA3E0FF123CEB0E
:100C3A00908000E07013301A101231E5906AF0EFDC
:100C4A00F0D3940040031211C8908002E07006901D
:100C5A008000E06005D218020BB2C218E4F5539086
:100C6A006940E06003020BB2301C15122F3D906AF6
:100C7A00F0EFF0D394004008301405E0FF12420B65
:100C8A00201B03020E91122DC0906AF0EFF0700340
:100C9A00020BB2906E48E060037401F0906B34E08E
:100CAA0054BF247F7003020D65147003020D46249D
:100CBA00026003020E3C201D077E247F4E1233E29F
:100CCA00906B0CE0FF7006906B10E06055906E3FE1
:100CDA00E0FEB50722A3E0FF906B0DE0B507189080
:100CEA006E41E0FF906B0EE0B5070C906E42E0FF9C
:100CFA00906B0FE06F602B906B10E06E7035906E0A
:100D0A0040E0FF906B11E0B50729906E41E0FF903B
:100D1A006B12E0B5071D906E42E0FF906B13E0B5D1
:100D2A000711C216906D357403F012002175510136
:100D3A00020E91906E3F74FFF0020E91906E37E0B2
:100D4A00FF906B36E06F6003020E91906E37E004FD
:100D5A00F0E4F551906D34F0020E91301603020E54
:100D6A0091906B35E0D3940A5003020E0FA3E0640E
:100D7A00026003020E0F906AFDE0FF906B3FE06F86
:100D8A006003020BB2906AFEE0FF906B40E06F6076
:100D9A0003020BB2906AFFE0FF906B41E06F6003C1
:100DAA00020BB2906B00E0FF906B42E06F600302AF
:100DBA000BB2906B01E0FF906B43E06F6003020B94
:100DCA00B2906B02E0FF906B44E06F6003020BB2DB
:100DDA007E247F5C1233E2906B3763A201906AF53E
:100DEA0063A2017F12122B45906B4963A201906E98
:100DFA003F63A2017F04122B45906D357406F0758E
:100E0A005102020BB27403446B7003020BB212421A
:100E1A003DD216E4F551906D34F0906E4304F0E43F
:100E2A00906E36F0A3F0201D5E7E247F651233E2B9
:100E3A008055301652906B34E020E74B906B36E0C9
:100E4A00FF906E36E0FE6F600D906E3EE07007EE2A
:100E5A00146F70338013906E36E004F0906AF0E0FD
:100E6A00FFD39404400312401D90683C7482F0A39F
:100E7A007401F0906B36E090683EF07E687F3C7DAE
:100E8A0003123BF7020BB2201603020F4D9080D0DB
:100E9A00E0700B906B08E0FEA3E0FF123CEBE5511B
:100EAA007066906E43E0D3943C4037906E3EE0709B
:100EBA0031120006906E437401F0E4906C34F0A392
:100ECA007412F0906E37E0906C36F0A374FDF090D7
:100EDA00694363A201906C3863A2017F12122B4509
:100EEA008006124084EF60207E6C7F34906C35E07F
:100EFA002404FD123BF7906E3EE06003020BB290B1
:100F0A006B14E0F551020BB212421AEF60159068A9
:100F1A003C7483F0E4A3F07E687F3C7D02123BF7C9
:100F2A00020BB2E55164016003020BB2906D34E02A
:100F3A0004F0E0C3940540B0C216E4A3F012002105
:100F4A00020BB2E55164016003020BB2906D35E009
:100F5A00147003020FF114700302101D14700302BF
:100F6A0010C514700302117B24FE60692406600315
:100F7A00020BB2E4F553F53C74EC253CF582E434FB
:100F8A0069F583E0FF74F5253CF582E4346AF5835C
:100F9A00EFF0053CE53CB43FDF202121906B0C6368
:100FAA00A201906E3F63A2017F04122B45906D351A
:100FBA007401F0906D34F0755103020BB2906D35E7
:100FCA007404F0906D347401F0755114906E3F748E
:100FDA00FFF0020BB2E4F553123ED7906D3574015F
:100FEA00F0755103020BB2906E3FE0600B906B08F4
:100FFA00E0FEA3E0FF123CEB755102906D357402DE
:10100A00F0906B03E07003020BB2906D357403F03D
:10101A00020BB2906E3FE070030210B6906C34740B
:10102A0080F0906C367402F0E4A3F0A304F0906AA6
:10103A00FD63A201906C3963A2017F0A122B4590CD
:10104A006C437430F0A3747BF0E4F53C746B253C7C
:10105A00F582E43469F583E0FF60117445253CF5B7
:10106A0082E4346CF583EFF0053C80E07445253C5E
:10107A00F582E4346CF583747DF07446253CF58280
:10108A00E4346CF583E4F0E53C2411906C35F07C93
:10109A006E7D3F906B08E0FAA3E0FB7F02123AF202
:1010AA007E6C7F34E53C2413FD123BF7906D35745A
:1010BA0004F0906B14E0F551020BB2906E3FE070B1
:1010CA000302116C906C347480F0906C367401F0E9
:1010DA00E4A3F0A304F0A37430F0A3747BF0E4F566
:1010EA003C746B253CF582E43469F583E0FF6011BA
:1010FA00743B253CF582E4346CF583EFF0053C80C3
:10110A00E0743B253CF582E4346CF583747DF0741D
:10111A003C253CF582E4346CF583E4F0E53C240795
:10112A00906C35F07C6E7D3F906B08E0FAA3E0FB93
:10113A007F02123AF27E6C7F34E53C2409FD123BB1
:10114A00F7906E3EE0601B12423DD216E4F55190D4
:10115A006D34F0906E4304F0E4906E36F0A3F00222
:10116A000BB2906D357404F0906B14E0F551020BDC
:10117A00B2906E3FE0FF6009F4600690800274103E
:10118A00F020212B755102906D34E06401FFF0A329
:10119A007401F0EF6005906B0C8003906B1063A2F2
:1011AA0001906E3F63A2017F04122B45020BB275B8
:0D11BA005114906E3F74FFF0020BB280FEE6
:0111C7002205
:1011C800906B35E0B444047F0180027F00906B345B
:1011D800E0B447047E0180027E00EE5F604A906AB8
:1011E800FDE0906B36F0906AFEE0906B37F0906A05
:1011F800FFE0906B38F0906B00E0906B39F0906BEB
:1012080001E0906B3AF0906B02E0906B3BF0906BD2
:10121800357452F0906AEA63A2019080A863A20133
:101228007F06122B450216D6906AF0E0C394085048
:10123800030216DF906AFDE0FF906B36E06F6003F3
:101248000216DF906AFEE0FF906B37E06F600302E2
:1012580016DF906AFFE0FF906B38E06F60030216BC
:10126800DF906B00E0FF906B39E06F60030216DFE0
:10127800906B01E0FF906B3AE06F60030216DF901D
:101288006B02E0FF906B3BE06F60030216DF906E2D
:1012980048E060037401F0906E497464F0906B3517
:1012A8007452F0906B34E0644D703C7E247F6F1272
:1012B80033E27E247F851233E212422E7E247FAAF7
:1012C8001233E27E247FBA1233E27E247FC61233C1
:1012D800E27E247FC81233E27E247FD11233E27E7D
:1012E800247FD31233E222906B34E0644C70527E38
:1012F800257F201233E2906B3CE0F53DA3E0F53EFC
:10130800E4F53F7D03AF3EAE3D1234C77E257F5BDB
:101318001233E2AE3DAF3EE4FB7D101235A57E24CC
:101328007FD11233E27410253EF53EE4353DF53D9C
:10133800053FE53FC3941040CA7E247FD11233E2B3
:1013480022906B34E0646C705CF5417E257F5E1200
:1013580033E2E4F540AF417E007D031234C77E25B9
:101368007F5B1233E2E4F53FA841E6FF743E253F78
:10137800F582E4346BF583EFF00541053FE53FB4B2
:1013880010E67E6B7F3EE4FB7D101235A57E247F40
:10139800D11233E20540E540C3940840B87E247F6B
:1013A800D11233E222906B34E0644B7046F53F74FF
:1013B80026253FF582E4346BF583E0FF6016743C24
:1013C800253FF582E4346BF583E0B50710053FE56A
:1013D8003FB408DB9069407432F00216D6906B3443
:1013E8007421F0301D030216D67E257F991233E250
:1013F8000216D6906B34E06452704E201D077E258D
:101408007FA11233E2906B3DE0906AF0F0E4F53F83
:10141800906AF0E0FDE53FC39D5022906B3CE025CB
:101428003F24EBF582E43469F583E0FF743E253F01
:10143800F582E4346BF583EFF0053F80D37E6B7F54
:1014480034ED240AFD123A6C22906B34E064497042
:1014580045201D077E257FAC1233E2906B3CE0F5FA
:101468003DA3E0F53EE4F53F853E82853D83E0FF00
:10147800743E253FF582E4346BF583EFF0053EE5D5
:101488003E7002053D053FE53FB480DC7E6B7F344E
:101498007D8A123A6C22906B34E064446003021532
:1014A8002F906B3CE0FF644470030216D6EFB43112
:1014B8000CC21D7E257FB41233E20216D6906B3C17
:1014C800E0B4300CD21D7E257FC01233E20216D65E
:1014D800906B3CE0B4320CD21E7E257FCD1233E2F5
:1014E8000216D6906B3CE0B4330CC21E7E257FDB1F
:1014F8001233E20216D6906B3CE0B4340CD21F7E55
:10150800257FEA1233E20216D6906B3CE0B4350C24
:10151800C21F7E257FF71233E20216D6906B3CE09D
:10152800FF12001E0216D6906940E07013201D07B6
:101538007E267F051233E2906B347421F00216D6B2
:101548009069407432F0906B34E0FFB45104C2AF3C
:1015580080FEEF64577045201D077E267F131233E7
:10156800E2906B3DE0906AF0F0E4F53F906AF0E0BD
:10157800FFE53FC39F40030216D6743E253FF58220
:10158800E4346BF583E0FF906B3CE0253F24EBF5FA
:1015980082E43469F583EFF0053F80D0906B34E046
:1015A80064536003021651201D077E267F1E1233E6
:1015B800E2906AFDE0FF9069F4E06F703C906AFE8B
:1015C800E0FF9069F5E06F7030906AFFE0FF906986
:1015D800F6E0B50724906B00E0FF9069F7E0B507E7
:1015E80018906B01E0FF9069F8E0B5070C906B026A
:1015F800E0FF9069F9E06F6016906B347421F03069
:101608001D030216D67E267F2D1233E20216D6E47B
:10161800F53FE4F55474EB253FF582E43469F5832E
:10162800E0FDAF3F1241B2053FE53FC394FE40E203
:10163800C2AFE4907FF0F0A3F0907FFD74AAF0A30E
:1016480074FFF0A37455F080FE906B34E0644F7023
:101658004B906B3CE0F53DA3E0F53EE53E453D7023
:101668000A201D077E267F361233E2201D077F2AB7
:101678007E001233E2E4F53F743E253FF582E43400
:101688006BF583E0853E82853D83F0053EE53E703F
:1016980002053D053FE53FB480DE8032906B34E0C3
:1016A800B4452B201D077E267F3D1233E2906B3C0C
:1016B800E0FFA3E0907FF0CFF0A3EFF0C2AF907F00
:1016C800FD74AAF0A374FFF0A37455F080FE7E6B3E
:0716D8007F347D08123A6C1B
:0116DF0022E8
:103FE500AE07EEC39430400BEED394395005EE2462
:103FF500D0FF22EEC39461400BEED394665005EEDC
:1040050024A9FF22EEC39441400BEED394465005FC
:08401500EE24C9FF22AF0622D0
:10288900C214E4906E48F0D221C217906E3EF090C7
:102899006AFD63A201906E3863A2017F06122B457F
:1028A900E4F53DE53D75F003A4246EF582E4342694
:1028B900F583E493FB740193FA740293F9121EF6FB
:1028C9007003022A69E4F53EF53FFD746B2DF5822C
:1028D900E43469F583E0FF7003022A64E53D75F08D
:1028E90003A4246EF582E43426F583E493FB740192
:1028F90093FA740293F9853E82758300121F0FFEC5
:10290900EFB50608753F01053E022A60E53F7003F1
:10291900022A60EE6003022A5BE53D24FE60221470
:102929007003022A4B147003022A4F147003022AFF
:102939005724046003022A64906E487401F0022A45
:1029490064D214746B2DF582E43469F583E0FF6475
:102959002D7003022A64123FE5EFC454F0FC746C35
:102969002DF582E43469F583E0FF123FE5EF2C9001
:102979006E38F0746D2DF582E43469F583E0FF1249
:102989003FE5EFC454F0FC746E2DF582E43469F52B
:1029990083E0FF123FE5EF2C906E39F0746F2DF54F
:1029A90082E43469F583E0FF123FE5EFC454F0FC9B
:1029B90074702DF582E43469F583E0FF123FE5EF89
:1029C9002C906E3AF074712DF582E43469F583E048
:1029D900FF123FE5EFC454F0FC74722DF582E43424
:1029E90069F583E0FF123FE5EF2C906E3BF07473BD
:1029F9002DF582E43469F583E0FF123FE5EFC45415
:102A0900F0FC74742DF582E43469F583E0FF123F1C
:102A1900E5EF2C906E3CF074752DF582E43469F580
:102A290083E0FF123FE5EFC454F0FC74762DF58284
:102A3900E43469F583E0FF123FE5EF2C906E3DF039
:102A49008019D2178015906E3E7401F0800DC22155
:102A59008009E4F53FF53E0D0228D4053D0228AC76
:012A6900224A
:03000300023E1AA0
:0D3E1A00C0E0C083C082C0D075D000C007DA
:103E2700C2A8908008E0FFEF54F06035EF30E40857
:103E3700D21A9080087410F0EF30E508D21C9080F9
:103E4700087420F0EF30E608D21B9080087440F029
:103E5700EF30E7069080087480F0908008E0FF80DC
:093E6700C690800874FFF0D2A897
:0B3E7000D007D0D0D082D083D0E03249
:103ED7009080007480F0906AF563A201F583F58203
:103EE70063A2017F08122B45906AFD63A2019080AF
:103EF7008863A2017F0A122B45906B07E0FF908031
:103F0700B1F09080E1EFF09080957455F0A3F090B8
:0C3F170080007401F09080097470F022AA
:043B7600AD07AC06E5
:103B7A00908009E04410F09080A0E0706F9080A1DE
:103B8A007482F09080A874FFF0A3F0A3F0A3F0AFC2
:103B9A0004AE079080AEEEF0AE05A3EEF0AE07904D
:103BAA0080ACEEF0AE05A3EEF09080007402F090C7
:103BBA006F681220B600000000906F68E0908040A5
:103BCA00F0906F69E0908041F0906F6AE0908042D7
:103BDA00F0906F6BE0908043F0A3E4F0A3F0A3F0C1
:0C3BEA00A3F0908018F0A3F0A3F0A3F06B
:013BF60022AC
:043CEB00AD07AC066F
:103CEF00908009E04440F09080D0E070559080D1F2
:103CFF007482F0AF049080DEEFF0AF05A3EFF09089
:103D0F0080027402F0906F6C1220B60000000090D9
:103D1F006F6CE0908058F0906F6DE0908059F0904C
:103D2F006F6EE090805AF0906F6FE090805BF0A321
:103D3F00E4F0A3F0A3F0A3F0908030F0A3F0A3F091
:023D4F00A3F0DF
:013D5100224F
:1038A800908009E04420F09080B8E0600302394934
:1038B8009080B97482F07F039080C6EFF07FCDA32B
:1038C800EFF07F039080C4EFF0A374CDF0300222B4
:1038D800906B0CE09080C0F0906B0DE09080C1F090
:1038E800906B0EE09080C2F0906B0FE09080C3F078
:1038F800800C9080C074FFF0A3F0A3F0A3F0908038
:10390800017402F0906F701220B600000000906FF2
:103918006CE090804CF0906F6DE090804DF0906F6F
:103928006EE090804EF0906F6FE090804FF0A3E4CF
:10393800F0A3F0A3F0A3F0908024F0A3F0A3F0A3E9
:01394800F08E
:01394900225B
:103AF2008C3D8D3EA907EAFDE975F018A424ACFFC0
:103B0200E5F034808F82F583EDF0EBFDE975F01876
:103B1200A4FFAEF024ACFBEE34808B82F583A3EDE0
:103B2200F0853E828C83E0FDEF24A8FFEE3480FE18
:103B32008F82F583EDF0853E828C83A3E08F828EA7
:103B420083A3F0853E82853D83A3A3E0FDE975F062
:103B520018A424A8FFE5F03480FE8F82F583A3A386
:103B6200EDF0853E828C83A3A3A3E08F828E83A394
:043B7200A3A3F022F7
:063A6C008D42AB07AA0623
:103A7200906F68E0FCA3E0FDA3E0FEA3E0F5468EB4
:103A8200458D448C43AE02AF038E838F8263A201C5
:103A9200E545540744C0F58385468263A201AF42DF
:103AA200122BAE908000E020E5F9E4FCFDFEE54635
:103AB2002542F546EE3545F545ED3544F544EC3500
:103AC20043F543C2A8908040E543F0A3E544F0A348
:103AD200E545F0A3E546F0D2A89080007420F0AF4F
:0F3AE20046AE45AD44AC43906F681220AAAF4288
:013AF10022B2
:063BF7008D3DAB07AA069C
:103BFD00906F6CE0FCA3E0FDA3E0FEA3E0F5418E29
:103C0D00408D3F8C3EAE02AF038E838F8263A20147
:103C1D00E540540744D0F58385418263A201AF3D51
:103C2D00122BAEE4FCFDFEE541253DF541EE3540A0
:103C3D00F540ED353FF53FEC353EF53EC2A89080A1
:103C4D0058E53EF0A3E53FF0A3E540F0A3E541F0D4
:103C5D00D2A89080027420F0AF41AE40AD3FAC3E93
:083C6D00906F6C1220AAAF3D1C
:013C7500222C
:0237FA008F3E00
:1037FC00908001E030E5037F0022906F70E0FCA325
:10380C00E0FDA3E0FEA3E0F5428E418D408C3F909D
:10381C006E3863A201E541540744C8F583854282A2
:10382C0063A2017F06122BC4E5422406F542E4355F
:10383C0041F541E43540F540E4353FF53F906D36B8
:10384C0063A201E541540744C8F58385428263A213
:10385C0001AF3E122BC4E4FCFDFEE542253EF542D1
:10386C00EE3541F541ED3540F540EC353FF53FC2C5
:10387C00A890804CE53FF0A3E540F0A3E541F0A310
:10388C00E542F0D2A89080017420F0AF42AE41AD79
:0B389C0040AC3F906F701220AAAF3EBE
:0138A70022FE
:1031E500C2A89081E0E0F53D053D053D053D053D65
:1031F500053D053D053D053D053D053D908010E03E
:10320500F540A3E0F541A3E0F542A3E0F543908145
:10321500E1E0F53D053D053D053D053D053D053D2A
:10322500053D053D053D053D908014E0F544A3E0D1
:10323500F545A3E0F546A3E0F547D2A8E546B54236
:1032450008E547B543037F0022E4F53DE54654070D
:1032550044E0F58385478263A201906B3463A20144
:103265007F08122BDC906B3663A201906AEA63A299
:10327500017F06122B45906B34E0F53EA3E0F53F48
:10328500E4F53D906B34E0702AA3E024F8F53DE5C4
:1032950046540744E0F58385478274082582F58204
:1032A500E43583F58363A201906B3463A201AF3DDE
:1032B500122BDCAE3EE4FCFDE547253FF547E54630
:1032C5003EF546ED3545F545EC3544F544C2A89047
:1032D5008014E544F0A3E545F0A3E546F0A3E547F2
:0B32E500F0D2A89080007440F0AF3DD4
:0132F00022BB
:102DC000C2A89081E6E0F53D053D053D053D053D88
:102DD000053D053D053D053D053D053D908028E04F
:102DE000F540A3E0F541A3E0F542A3E0F54390816F
:102DF000E7E0F53D053D053D053D053D053D053D4E
:102E0000053D053D053D053D90802CE0F544A3E0E2
:102E1000F545A3E0F546A3E0F547D2A8E4F53DE586
:102E200046B5420AE547B54305C21B022F1EE546DB
:102E3000540744F0F58385478263A201906B3463A5
:102E4000A2017F08122BDC906B34E0F53EA3E0F585
:102E50003FE53F453E70099080027410F07F0022EC
:102E6000906E3FE0FFF4602D906B36E06F707690CF
:102E70006E40E0FF906B37E06F706A906E41E0FF4C
:102E8000906B38E06F705E906E42E0FF906B39E0BF
:102E90006F60228050906B36E0906E3FF0906B3701
:102EA000E0906E40F0906B38E0906E41F0906B399E
:102EB000E0906E42F0906B34E0702AA3E024F8F5C5
:102EC0003DE546540744F0F5838547827408258222
:102ED000F582E43583F58363A201906B3463A2012C
:102EE000AF3D122BDCAE3EE4FCFDE547253FF54748
:102EF000E5463EF546ED3545F545EC3544F544AF40
:102F000043AE42AD41AC40AB47AA46A945A844D325
:102F100012209940099080027410F07F0022C2A80C
:102F200090802CE544F0A3E545F0A3E546F0A3E549
:0C2F300047F0D2A89080027440F0AF3D42
:012F3C002272
:102F3D00C2A89081E3E0F53D053D053D053D053D0C
:102F4D00053D053D053D053D053D053D90801CE0DC
:102F5D00F540A3E0F541A3E0F542A3E0F5439081F0
:102F6D00E4E0F53D053D053D053D053D053D053DD2
:102F7D00053D053D053D053D908020E0F544A3E070
:102F8D00F545A3E0F546A3E0F547D2A8E4F53DE508
:102F9D0046B5420AE547B54305C21C023085E546F4
:102FAD00540744E8F58385478263A2019068406326
:102FBD00A2017F0E122BF2906840E0F53EA3E0F5E2
:102FCD003F906E38E0FF906848E06F706C906E39FE
:102FDD00E0FF906849E06F7060906E3AE0FF906896
:102FED004AE06F7054906E3BE0FF90684BE06F705D
:102FFD0048906E3CE0FF90684CE06F703C906E3DE9
:10300D00E0FF90684DE06F7030906840E0702AA34B
:10301D00E024F2F53DE546540744E8F58385478203
:10302D00740E2582F582E43583F58363A2019068E1
:10303D004063A201AF3D122BF2AE3EE4FCFDE5472D
:10304D00253FF547E5463EF546ED3545F545EC356D
:10305D0044F544AF43AE42AD41AC40AB47AA46A99F
:10306D0045A844D31220995006E53F453E7009907E
:10307D0080017410F07F0022C2A8908020E544F0FA
:10308D00A3E545F0A3E546F0A3E547F0D2A890806F
:06309D00017440F0AF3D9C
:0130A300220A
:0433E2008E438F4443
:1033E600906F68E0FCA3E0FDA3E0FEA3E0F54A8E43
:1033F600498D488C47E54AFFE5495407FEE42FF519
:1034060046EE34C0F545854682F5837423F00546BD
:10341600E546700205455345C7F582854583740A1E
:10342600F00546E546700205455345C7906AFD63BB
:10343600A20185458385468263A2017F06122BAED3
:1034460074062546F546E43545F5458543838544AA
:103456008263A20185458385468263A201122B926F
:10346600908000E020E5F9E4FCFDFE906F68E0F84E
:10347600A3E0F9A3E0FAA3E02FFFEE3AFEED39FD53
:10348600EC38FCEF2408FFE43EFEE43DFDE43CFCA2
:10349600906F681220AAC2A8906F68E0908040F0F2
:1034A600906F69E0908041F0906F6AE0908042F002
:1034B600906F6BE0908043F0D2A89080007420F06B
:0134C60022E3
:0635A5008E438F448D45AA
:1035AB00906F68E0FCA3E0FDA3E0FEA3E0F54B8E7B
:1035BB004A8D498C48E54BFFE54A5407FEE42FF54D
:1035CB0047EE34C0F546854782F5837423F00547F3
:1035DB00E547700205465346C7F582854683EBF0F7
:1035EB000547E547700205465346C7906AFD63A23F
:1035FB000185468385478263A2017F06122BAE7439
:10360B00062547F547E43546F546854383854482D1
:10361B0063A20185468385478263A201AF45122BC6
:10362B00AE908000E020E5F974082545F545FFE4F0
:10363B00FCFDFEE54B2FF54BEE354AF54AED3549D2
:10364B00F549EC3548F548C2A8908040E548F0A311
:10365B00E549F0A3E54AF0A3E54BF0D2A890800032
:10366B007420F0AF4BAE4AAD49AC48906F68122056
:01367B00AAA4
:01367C00222B
:0634C7008E428F43AB05AD
:1034CD00906F68E0FCA3E0FDA3E0FEA3E0F5498E5C
:1034DD00488D478C46E549FFE5485407FEE42FF536
:1034ED0045EE34C0F544854582F5837423F00545DA
:1034FD00E545700205445344C7F582854483EBF0DE
:10350D000545E54570020544906AFD63A2018544B9
:10351D008385458263A2017F06122BAE7406254575
:10352D00F545E43544F5445344C7E5428545828568
:10353D004483F00545E545700205445344C7F582C3
:10354D00854483E543F00545E54570020544534444
:10355D00C7908000E020E5F9E549240AF549E435F6
:10356D0048F548E43547F547E43546F546C2A89099
:10357D008040E546F0A3E547F0A3E548F0A3E54913
:10358D00F0D2A89080007420F0AF49AE48AD47ACA2
:07359D0046906F681220AA9E
:0135A4002204
:10415C00E5D220E0FBC2AF438E2075D2028F827570
:0C416C008300E0FFE4F5D2538EDFD2AFF9
:014178002224
:1041B200E5D220E0FBC2AF43D2028F82758300EDCD
:0A41C200F075D25063D250D2AF2244
:103C7600E4FEEE04FF12415C74F52EF582E4346A2C
:103C8600F583EFF00EBE3FEAE4FEEE247FFF12411D
:103C96005C746B2EF582E43469F583EFF0746B2E59
:103CA600F582E43469F583E0701B746B2EF582E4CB
:103CB6003469F5837420F0746C2EF582E43469F56A
:103CC60083E4F080040EBE80C1E49069EAF0FEAFA2
:103CD6000612415C74EB2EF582E43469F583EFF04D
:043CE6000EBEFEEB25
:013CEA0022B7
:10417900A2AF9227C2AF8C838D82EF122C0A43A281
:0C41890020122C0C53A2DFA22792AFFFE3
:014195002207
:024114008F3DDD
:10411600A2AF9227C2AFE4F5838D827406122C0AF1
:10412600E53D43A220122C0C53A2DFA22792AF7FBB
:014136000187
:014137002265
:024138008F3DB9
:10413A00A2AF9227C2AFE4F5838D82740A122C0AC9
:10414A00E53D43A220122C0C53A2DFA22792AF7F97
:01415A000163
:01415B002241
:102A6A00A907E7FFA805EF93C3966008403B74FCEB
:102A7A002FFF80F00F08EF93C3966008402B74FB7A
:102A8A002FFF80E00F08EF93C3966008401B74FA8B
:102A9A002FFF80D00F08EF93D3966008400B74F98C
:102AAA002FFF80C01F1F1F1F1FEF54FEF80303F7DD
:102ABA00E893FC08E893FD08E893FE08E893FF22F0
:102ACA0009E993C39D6008402974FB29F980F1093B
:102ADA00E993C39E6008401A74FA29F980E209E969
:102AEA0093D39F6008400B74F929F980D3191919F7
:102AFA001919E9C313C313FF22740093F8ECC3989E
:102B0A004024701F740193F8EDC39840197014742F
:0E2B1A000293F8EEC398400E7009740393F80E
:102B2800EFC39840037F00227F0122EDF8E6F0080A
:102B3800A3DFFA22EDF8E0F608A3DFFA22E0A363A8
:102B4800A201F0A363A201DFF475A20022E0A3634F
:102B5800A201F0A363A201E0A363A201F0A363A210
:102B680001E463A201F0A363A201DFE175A20022E0
:102B7800E0A363A2016DFE936CFDEE058393FC1543
:102B88008363A201DFEA75A200227F00E493A363B6
:102B9800A201F00F600CA3E583C2E3F58363A201F1
:102BA80080EA75A20022E0A363A201F0A3E583C234
:102BB800E3F58363A201DFEE75A20022E0A363A21E
:102BC80001F0A3E583C2E4D2E3F58363A201DFEC5D
:102BD80075A20022E583C2E3F583E0A363A201F0B6
:102BE800A363A201DFEE75A20022E583C2E4D2E36B
:102BF800F583E0A363A201F0A363A201DFEC75A251
:102C08000022F922C002C004C00612FFF0D006D08C
:042C180004D00222C0
:103F660020536572763A0020547261737353656EFE
:103F7600644552520A00205265496E6974204341D5
:103F86004E0A002043414E283029203E20544F211E
:103F96000A0020545520300A0020545520310A00CA
:03001E00E4FF22DA
:1040B700C28DC2AF438901C28C906E5EE0FF70076C
:1040C700F58A758CEE8016EFB40508E4F58A758CD1
:1040D700B8800AEFB40A06E4F58A758C70D28CD2E0
:0240E700AF2206
:103FA600C28DC2AF438901C28C906E5EE0FF701471
:103FB600302609F58A758CDCC226801E758A6675E0
:103FC6008CFC8016EFB40508E4F58A758CEE800A41
:0F3FD600EFB40A06E4F58A758CDCD28CD2AF22E8
:10419600123D52124243D225E4F537906F66F0F590
:0C41A60025F53B1240B7C226E4F5392293
:10401D00EF24FCF53D201D127E3F7F661233E27EBC
:10402D006B7F387B01AD3D1235A5906B3863A201D6
:10403D00906EE663A201AF3D122B45853D25E4F55B
:03404D0036C22355
:01405000224D
:0F420B00D3EF6480948E5006E53B70028F3B2208
:10268300208D0302271FC28C202503022778E5250E
:10269300605474EA2536F582E4346EF583E024054C
:1026A300F53DD3940E4008E4F525D2230227787430
:1026B300E62536F582E4346EF5837D27AF3D122B94
:1026C3003CE53D2536F536E52730E702D2261240B4
:1026D300B7123E7BE536C395255003022778E4F510
:1026E30025D223022778E5386014906E4A7D27FFB0
:1026F300122B3C1240B7123E7BE4F5388077E53B62
:1027030060149068407D27FF122B3C1240B7123EA5
:102713007BE4F53B805F123DB71240B71230A48FC4
:102723003DEF6051123FA6E4F539E53AC3946E508C
:1027330018745F253AF582E4346EF583E53D253A56
:10274300F53A7D27AF3D122B33301424E52730E7CC
:102753000330021C906D367D27AF3D122B33AF3D06
:102763001237FAEF700A201D077E3F7F6D1233E2A6
:10277300AF3D1221A030201230130D0539E539D3B6
:1027830094F04004C2AF80FEC220201503022885C6
:10279300E5376031D39401400415378028906F6684
:1027A300E004F0E0D39403400D201D077E3F7F7CBF
:1027B3001233E2124196201D077E3F7F891233E2D6
:1027C300E4F537D225302443E538703F906E4A0450
:1027D300F0A37408F0A37480F0A37401F0A374064B
:1027E300F0906EE1E0906E4FF0906EE2E0906E50EC
:1027F300F0906EE3E0906E51F0906EE4E0906E52D4
:10280300F0E4A3F0A3F075380BC224302272906E6B
:10281300DFE07035E5387031906E4A7442F0A3748E
:1028230008F0906EE0E0906E4CF0906EE5E0906EF4
:102833004DF0A37401F0753806201D077E3F7F9885
:102843001233E2906EDFE004F0906EDFE06402701A
:102853002FE538702B906E4A7402F0A37408F09041
:102863006EE0E0906E4CF0A3F0A37401F0753806AF
:10287300201D077E3F7F9F1233E2906EDFE004F05E
:05288300C21512002641
:01288800222D
:10408400E53A602CE4906C34F0A3E53AF0906E3796
:10409400E0906C36F0A37419F0906E5F63A2019007
:1040A4006C3863A201AF3A122B45E4F53A7F012242
:0340B4007F002268
:0B421A00302305C2237F01227F002219
:0100210022BC
:06423D00E4F53AF525222C
:100006007F01E4906943F0A3F0A3F0FEEF25E0FF43
:040016000EBE08F81A
:01001A0022C3
:1040E9002043616E457247495400200A00204B560F
:1040F90054210A002043616E457272434821000A27
:0B410900000A2052657145727221000F
:1030A400E59B541F6020201D1A7E407FE91233E205
:1030B400E59B541FFF7E007D031234C77E407FF3DF
:1030C4001233E2E4F59BE5BA30E010E4F5B375B1F0
:1030D40080F5B2D225F537906F66F0E5CFF4700332
:1030E4000231E2753F01E4F53EE5CFF4553F70034C
:1030F4000231D0E53EC454F0F5B1E5B2547F64200A
:103104006003023192E5B3540FF52B85BC272002EE
:1031140016E5BD541FFF131313541FFFE5BD54E000
:1031240044184FF5288006E5BD54E0F528E5BDC4F4
:103134003354E0FFE5BE131313541F4FF529E5BEC6
:10314400C43354E0FFE5BF131313541F4FF52A850E
:10315400A32C85A32D85A32E85A32F85A33085A31A
:103164003185A33285A333E4F5B230020C85AE3445
:1031740085AF3575B3D07F0F22E527547EB527057B
:1031840075B350800375B3D0E52B2405FF22E5B257
:1031940030E60A201D077E407FF61233E2E5B25482
:1031A4009F6023201D207E407FFD1233E2AFB27E5C
:1031B400007D031234C7AFB37E007D031234C77E93
:1031C400417F081233E2E4F5B275B3D0E53F25E060
:1031D400F53F053EE53EC3940850030230ED7F0001
:0131E40022C8
:103E7B0020025875B180E4F5B3F5B28527BCE5296E
:103E8B00C4135407FFE52854E04FF5BDE529333340
:103E9B003354F8FFE52AC41354074FF5BEE52A3314
:103EAB00333354F8F5BF852CA3852DA3852EA3851D
:103EBB002FA38530A38531A38532A38533A3E52BAF
:0C3ECB00540F2450F5B375370AC22522AD
:103DB70020025F75B190E5B220E613201D107E4109
:103DC7007F0A1233E2AFB27E007D031234C7E4F5F7
:103DD700B3F5B274862515F582E43461F583E0F511
:103DE700BCE4F5BD74872515F582E43461F583E0FD
:103DF700FF33333354F8F5BE75BF780515051574D1
:103E0700862515F582E43461F583E07002F51575B2
:033E1700B3502283
:09422500EF6003C29622D296223A
:103D520043AB01C2E8C2EAE4FFEFC454F0F5B1C3D9
:103D6200EF64809488500575B3D08003E4F5B3E422
:103D7200F5B2F5BCF5BDF5BEF5BFF5C4F5C5F5C6A2
:103D8200F5C7F5A3F5A3F5A3F5A3F5A3F5A3F5A34D
:103D9200F5A30FBF0EC3906E5EE0FF25E0F5B4758C
:103DA200B50C75B66C75A11275AB0275C13E75C3C3
:043DB200FF75C203D4
:013DB60022EA
:101BAD00C7E0E3F0F3E7EEF7EDFBE920EEE1F0E05F
:101BBD00E73A20CACF20C8F1E5F2FC28C3F0E0EDEA
:101BCD00E8F22DC029207620312E30340A005452EF
:101BDD00414E5A004D415842005254530044454C19
:101BED004159004D4F4445004B5000545500434161
:101BFD004E004B5654004154004449520043414E4F
:101C0D004D4F4E00475254494D45005449545300D1
:101C1D005453494E5600000A41734F55543A200013
:101C2D0054530A005455204F4B0A00545520446913
:101C3D0061670A005455205265710A0020545520E1
:101C4D0054696D654F5554210A004154636F6E6E92
:101C5D006563740A000A4173494E3A20000A4352E3
:101C6D0043204552523A20000A4E6B703A20000A2A
:101C7D00CFF0E8EDFFF2E020EAEEECE0EDE4E0205D
:101C8D00D2D320002020D2D320E7E0EDFFF2EE21C9
:101C9D000A000ACDE520EFEEEDFFEB20F2E8EF2094
:101CAD00EFE0EAE5F2E0210A000011233246576524
:101CBD00748C9DAFBECADBE9F8100133225647750F
:101CCD00649C8DBFAEDACBF9E82130021367764400
:101CDD0055ADBC8E9FEBFAC8D931201203776654EF
:101CED0045BDAC9E8FFBEAD8C942536170041527E0
:101CFD0036CEDFEDFC8899ABBA52437160140537CF
:101D0D0026DECFFDEC9889BBAA63724051253406BF
:101D1D0017EFFECCDDA9B88A9B73625041352416AE
:101D2D0007FFEEDCCDB9A89A8B8495A7B6C2D3E197
:101D3D00F008192B3A4E5F6D7C9485B7A6D2C3F18E
:101D4D00E018093B2A5E4F7D6CA5B48697E3F2C07F
:101D5D00D129380A1B6F7E4C5DB5A49687F3E2D06E
:101D6D00C139281A0B7F6E5C4DC6D7E5F48091A35F
:101D7D00B24A5B69780C1D2F3ED6C7F5E49081B34E
:101D8D00A25A4B79681C0D3F2EE7F6C4D5A1B0823F
:101D9D00936B7A48592D3C0E1FF7E6D4C5B1A0922E
:101DAD00837B6A58493D2C1E0F0089129B24AD364A
:101DBD00BF48C15AD36CE57EF78108931AA52CB79D
:101DCD003EC940DB52ED64FF76028B109926AF348D
:101DDD00BD4AC358D16EE77CF5830A9118A72EB57D
:101DED003CCB42D950EF66FD74048D169F20A9326D
:101DFD00BB4CC55ED768E17AF3850C971EA128B35D
:101E0D003ACD44DF56E960FB72068F149D22AB304C
:101E1D00B94EC75CD56AE378F1870E951CA32AB13C
:101E2D0038CF46DD54EB62F97008811A932CA53E2C
:101E3D00B740C952DB64ED76FF89009B12AD24BF1C
:101E4D0036C148D35AE56CF77E0A8318912EA73C0C
:101E5D00B542CB50D966EF74FD8B029910AF26BDFC
:101E6D0034C34AD158E76EF57C0C851E9728A13AEC
:101E7D00B344CD56DF60E972FB8D049F16A920BBDC
:101E8D0032C54CD75EE168F37A0E871C952AA338CC
:101E9D00B146CF54DD62EB70F98F069D14AB22B9BC
:101EAD0030C74ED55CE36AF1780008040C020A06CF
:101EBD000E0109050D030B070FFF1BDBFF1BE1FFD8
:101ECD001BE6FF1BEAFF1BF0FF1BF5FF1BF8FF1BBB
:101EDD00FBFF1BFFFF1C03FF1C06FF1C0AFF1C1151
:091EED00FF1C18FF1C1DFF1C2343
:1041E300EF540F901EB693FEC454F0FEEFC4540F69
:0441F300932EFF22E6
:08422E007E1B7FAD1233E2227A
:0300230002367D25
:0B367D00C0E0C083C082C0D075D01830
:10368800309852C298755201AF9920074820030B11
:10369800EF64027040D203D291803A300C04C20C1D
:1036A8008024BF0904D20C802CBF0205530C8080F3
:1036B80024BF0312906613E50CF0630C80530C8052
:1036C800C203C291800F7436250CF582E43466F586
:1036D80083EFF0050C30995F30045A906185E0FF64
:1036E800E50DC39F4008C204D211C2908047D29012
:1036F800AF0D050D74362FF582E43467F583E0F5D8
:1037080010300B1953107F30012830D008300622B2
:10371800631080801D20061A631080801530011206
:10372800E50B5210300606A2D0929B8005A2D0B3BA
:07373800929B851099C299D4
:09373F00D0D0D082D083D0E0325A
:1016E000C20EE4906402F0906838F0D20DC202C2DB
:1016F00005906836F0A37478F0D20AE4906E5EF03C
:10170000906F7C7461F0A37486F0906F7CE475F048
:1017100001121F9185F082F58374C4F0906F7CE410
:1017200075F001121F9185F082F583E4F0906F7CD3
:1017300075F001121F9185F082F58374C4F0906FEB
:101740007CE475F001121F9185F082F5837401F03D
:10175000906F7CE475F001121F9185F082F583741F
:10176000C8F0906F7CE475F001121F9185F082F54E
:1017700083E4F0906F7C75F001121F9185F082F583
:101780008374C8F0906F7CE475F001121F9185F0AE
:1017900082F5837401F0906F7CE475F001121F9163
:1017A00085F082F58374C2F0906F7CE475F00112CD
:1017B0001F9185F082F583E4F0906F7C75F0011243
:1017C0001F9185F082F58374C2F0906F7CE475F010
:1017D00001121F9185F082F5837401F0906F7CE413
:1017E00075F001121F9185F082F583E4F0906F7C13
:1017F00075F001121F9185F082F583E4F0F51590E4
:101800006F74F0906F74E075F003A424C6F582E461
:10181000341EF583E493FB740193FA740293F91276
:101820001EF67003021BACE4906F76F0A3F0906F8D
:1018300075F0906F75E0246BF582E43469F583E010
:10184000FF7003021BA3906F74E075F003A424C61D
:10185000F582E4341EF583E493FB740193FA740279
:1018600093F9906F76E0F582758300121F0FFEEFFB
:10187000B5060F906F777401F0906F76E004F00278
:101880001B9A906F77E07003021B9AEE6003021BB5
:1018900091906F74E0B40F004003021BA39018A452
:1018A000F82828730218D102191E021A35021A3AB2
:1018B000021A69021AD0021BA3021A9F021BA3027A
:1018C0001B01021B55021B85021B89021BA3021B65
:1018D0008D906F75E0246BF9E43469FA7B01C003E5
:1018E0001B8B40754100754200E4F543D003122C78
:1018F0001C906F781220AA906F78E0F8A3E0F9A30B
:10190000E0FAA3E0FB7F007E8C7D0A7C00121FE3DF
:1019100012207590683AEEF0A3EFF0021BA3906FCF
:101920007C7461F0A37486F0906F75E0246BF5828F
:10193000E43469F583E024D0F515C394014007E54C
:1019400015D394084003E4F515E5156028906F7CE5
:10195000E475F001121F9185F082F58374C4F015CF
:1019600015906F7CE475F001121F9185F082F5836C
:10197000E515F080D4906F75E0246CF582E434694D
:10198000F583E024D0F515C394014007E515D39401
:10199000084003E4F515E5156028906F7CE475F0C8
:1019A00001121F9185F082F58374C8F01515906FB0
:1019B0007CE475F001121F9185F082F583E515F046
:1019C00080D4906F75E0246DF582E43469F583E08E
:1019D00024D0F515C394014007E515D394084003BE
:1019E000E4F515E5156028906F7CE475F001121F91
:1019F0009185F082F58374C2F01515906F7CE475C3
:101A0000F001121F9185F082F583E515F080D490E6
:101A10006F7CE475F001121F9185F082F583E4F08C
:101A2000906F7C75F001121F9185F082F583E4F0D0
:101A3000F515021BA3D20F021BA3906F75E0246B58
:101A4000F9E43469FA7B01C0031B8B4075410075D2
:101A50004200E4F543D003122C1C906F781220AAA8
:101A6000906F7BE0F509021BA3906F75E0FF246B7C
:101A7000F582E43469F583E0B43702D20B746C2F3D
:101A8000F582E43469F583E0FFB44E04C2018002BC
:101A9000D201EF64456003021BA3D206021BA39090
:101AA0006F75E0246BF9E43469FA7B01C0031B8B8A
:101AB00040754100754200E4F543D003122C1C90A0
:101AC0006F781220AA906F7BE0906E5EF0021BA3ED
:101AD000906F75E0246BF9E43469FA7B01C0031B55
:101AE0008B40754100754200E4F543D003122C1C75
:101AF000906F781220AA906F7BE0906402F0021B36
:101B0000A3906F75E0246BF9E43469FA7B01C0039C
:101B10001B8B40754100754200E4F543D003122C45
:101B20001C906F781220AAE4FFFEFDFC906F78E015
:101B3000F8A3E0F9A3E0FAA3E0FBD3122099400F49
:101B4000906F7AE0FFA3E0906836CFF0A3EFF0D279
:101B50000EC20D804E906F75E0246BF9E43469FA83
:101B60007B01C0031B8B40754100754200E4F543C7
:101B7000D003122C1C906F781220AA906F7BE090FB
:101B80006838F0801ED202801AD2058016C20A8000
:101B900012E4906F77F0906F76F0906F75E004F03C
:0C1BA000021832906F74E004F002180389
:011BAC002216
:1032F100C222C210C209C208906182740AF0E4902D
:103301006839F0906837E024F9FE906836E034FFC0
:10331100906300F0A3CEF0E4906184F0C212906655
:10332100157405F0C224E4F508906941E064557014
:1033310004A3E06481603BE4FF7F409061B6E4F068
:10334100A3DFFCE4FF7F20906616E4F0A3DFFCE43A
:10335100FF74032FF582E43466F583E4F0740B2FD8
:10336100F582E43466F583E4F00FBF08E4E4F50E7A
:10337100F50FE4F514F5139062FFF09062FEF0C2D0
:1033810004C211C207C203C20CF50D906185F0F5AC
:1033910009F50CF552C200C20BC20F90683A74FFD6
:1033A100F0A374F4F0750BFF1216E0C2ADE4F5C999
:1033B100D2CDD2CCC2C9C2CAF5CDF5CC90683AE023
:1033C100F5CBA3E0F5CA85CBCD85CACCD29ED29CE4
:1033D100D2CAC2ACC298C29975B81075B710D2AC36
:0133E10022C9
:1041F700E5126FFF901DB6936511F512EF901CB68F
:0342070093F5111B
:01420A002291
:023748008F43AD
:10374A00E4FC754461754500F512F511FDEDC3956C
:10375A004350170545E545AE447002054414F58209
:10376A008E83E0FF1241F70D80E30545E545AE443F
:10377A007002054414F5828E83E512F08545828530
:10378A004483E511F0054305437E677F367544613E
:10379A007545008F828E837402F00FBF00010E0CF4
:1037AA00E4FDEDC395435038854582854483E0F9AD
:1037BA0064026008E964036003B9090D8F828E838D
:1037CA007409F00FBF00010E0C8F828E83E9F00F8F
:1037DA00BF00010E0C0545E545700205440D80C287
:0F37EA008F828E837403F00FBF00010E0CAF04AB
:0137F90022AD
:03424300C207228D
:103F23008F4220043D300D3AAF42123748906185ED
:103F3300EFF0201D127E1C7F241233E27E617F008E
:103F4300E4FBAD421235A5300F057F01124225E592
:103F5300096003F54F22E4F50DD204C2992099FDBF
:033F6300D29922CE
:0221A0008F3E70
:1021A200906402E07003022444E52724BE70030217
:1021B20023ED24FA700302237124046003022444F1
:1021C200E52830E70302225CE52A6068E529C3942A
:1021D200024003022444E5297007E52A14F53F80F2
:1021E20006E52A241FF53FE53F75F004A42402F515
:1021F20082746335F0F5837D2C7F04122B33E53F27
:1022020075F004A424FEF582746135F0F5837D3007
:102212007F04122B3374F62529F582E43461F583A9
:102222007481F074B6253FF582E43461F58374015C
:10223200F0D2082274032529F582E43466F583740A
:1022420080F0E52975F004A42416F582746635F051
:10225200F5837D2C7F04122B3322E52B6408600367
:10226200022444E529C394044003022444201D07A8
:102272007E1C7F2D1233E2753E01E52A5407FFE5ED
:102282003EA807088002C333D8FCF53E7408250F28
:10229200F50FB50E067408250EF50EE52A547FFFDC
:1022A200E529C43354E02FFE7400250FF582E4348F
:1022B20060F583EEF0E52AC394805022EF131313E6
:1022C200541FFFE52925E025E02F2416F582E4348A
:1022D20066F583E0FFE53EF4FEEF5EF0802EE52A30
:1022E200547FFF131313541FFFE52925E025E02F28
:1022F2002416F582E43466F583E0453EF074002549
:102302000FF582E43460F583E04480F07401250F18
:10231200F582E43460F5837D2C7F04122B33E531A2
:10232200FEE530FF7C007D0A121F3CEF7405250F8D
:10233200F582E43460F583EFF07406250FF582E44C
:102342003460F583E532F07407250FF582E43460DA
:10235200F583E533F0301D030224447400250FF5A4
:1023620082E43460AF82FEE4FB7D081235A522E5EB
:102372002A54E064407003022444E529701DE52AD2
:102382001313543FFF7401A807088002C333D8FC1B
:1023920042139062FEE04513F08024E52964016057
:1023A20003022444E52A1313543FFF7401A80708CB
:1023B2008002C333D8FC42149062FFE04514F0E57A
:1023C2002975F020A4FFE52A547F7C002FFFEC350D
:1023D200F0FEEF25E0FFEE33FE74032FF582746406
:1023E2003EF5837D2CAF2B122B3322E52AB4011349
:1023F200201D077E1C7F311233E2E52D04906F67AA
:10240200F0C222E52AB40216240BF582E43466F502
:1024120083E52DF0201D077E1C7F381233E2E52A6A
:10242200B4031F240BF582E43466F583E52DF02016
:102432001D077E1C7F411233E2302206906EDF744C
:0224420002F0A6
:012444002275
:10002600906402E07003020A19301361050A9066B3
:1000360015E0600214F0906839E0600214F09068F0
:1000460038E06008906182E0600214F0C213300E5E
:1000560021906836E0FEA3E0FFD3906301E09F9015
:100066006300E09E500CA3E004F07006906300E08D
:1000760004F0302218906183E004F0E0D3940A4043
:100086000C201D077E1C7F491233E2C222E54FB4C5
:10009600010EE4F54FF50DD204C2992099FDD299CF
:1000A60030040DE50AD394064009C204D211800338
:1000B600E4F50A200E03020191906837E024FBFF65
:1000C600906836E034FFFEC3906301E09F906300C2
:1000D600E09E4012906184E0700CC20DFF12422532
:1000E6009061847401F0906837E024FDFF906836D3
:1000F600E034FFFEC3906301E09F906300E09E4002
:1001060012906184E0B4010B7F0112422590618454
:100116007402F0906837E024FEFF906836E034FF02
:10012600FEC3906301E09F906300E09E405D200463
:100136005A9067367441F0A37454F0A37424F0A364
:100146007443F0A3744FF0A314F0A3F0A37445F026
:10015600A37443F0A37454F0A3740DF0A3740AF0CF
:10016600906185740CF0E4F50DD204C2992099FDD6
:10017600D299E4906300F0A3F0906184F0301D03FF
:10018600020A197E1C7F571233E22230110AC2116D
:10019600300F05E4FF124225300403020678E54FCE
:1001A6006003020678200D03020678906182E06003
:1001B60003020678906838E06007E4906182F08078
:1001C60006906182740AF0301229C212E49061002E
:1001D600F0A37408F0906402E0906102F090661457
:1001E600E0906103F0A374FEF0A3748FF07F061213
:1001F6003F2322906F67E0FF6025E4906100F0A343
:100206007408F0906402E0906102F0A37483F0A396
:10021600EFF0E4A3F0906F67F07F06123F2322E52C
:100226000F650E7003020326906839E0600302042E
:1002360012E50E2408F53EE4906100F0A37408F080
:10024600906402E0906102F0A374F0F0A37406F0EB
:10025600A37491F07406253EF582E43460F583E0DC
:10026600906106F07407253EF582E43460F583E07C
:10027600906107F07401253EF582E43460F583E071
:10028600906108F07402253EF582E43460F583E05F
:10029600906109F07403253EF582E43460F583E04D
:1002A60090610AF07404253EF582E43460F583E03B
:1002B60090610BF07400253EF582E43460F583E02E
:1002C600FF547FFEC39440500BEFC454F00490617A
:1002D6000CF080167400253EF582E43460F583E068
:1002E600FFC454F0240590610CF07400253EF5829D
:1002F600E43460F583E0FFEEC4540F90610DF0EF37
:100306005480FF7405253EF582E43460F583E02FC2
:1003160090610EF09068397414F07F0F123F23221B
:10032600300973906603E0D39400406AE49061005C
:10033600F0A37408F0906402E0906102F0A37441A7
:10034600F0A37420F0754061754105E4F53E74161E
:10035600253EF582E43466F583E0F53F300A06FF74
:100366001241E38F3F854182854083E53FF0F4FFEC
:10037600E5822408F582E43583F583EFF00541E54F
:100386004170020540053EE53EC3940840C07F1516
:10039600123F23C20922301073906605E0D3940001
:1003A600406AE4906100F0A37408F0906402E09063
:1003B6006102F0A37445F0A37420F07540617541A5
:1003C60005753E087416253EF582E43466F583E02D
:1003D600F53F300A06FF1241E38F3F854182854093
:1003E60083E53FF0F4FFE5822408F582E43583F5E2
:1003F60083EFF00541E54170020540053EE53EC349
:10040600941040C07F15123F23C210222008030219
:1004160005159061F7E0FF9061F6E04F5401D39423
:10042600005003020515E4F53E74B6253EF582E458
:100436003461F583E0700302050774B6253EF58244
:10044600E43461F583E4F0906100F0A37408F09061
:100456006402E0906102F0A374F0F0A37403F0A3C9
:100466007491F0E53EC4540F2408A3F0E53E540F02
:10047600A3F0E53E25E025E0F53E24FEF582E434D2
:1004860061F583E0906108F074FF253EF582E4345F
:1004960061F583E0906109F07400253EF582E4344D
:1004A60062F583E090610AF07401253EF582E4343A
:1004B60062F583E090610BF0E4A3F07402253EF54B
:1004C60082E43463F583E090610DF07403253EF514
:1004D60082E43463F583E090610EF07404253EF502
:1004E60082E43463F583E090610FF07405253EF5F0
:1004F60082E43463F583E0906110F07F11123F23AC
:1005060022053EE53EC39440500302042FC20890E4
:100516006615E0704130053E7478F0E4906100F0B5
:10052600A37408F0906402E0906102F0A374F0F006
:10053600E4A3F0A37490F0A37408F0E4A3F0A3F08E
:10054600A3F0A3F0A3F0A3F0A3F0A3F0A3F0A3F00D
:100556007F11123F2322E508C394045070E5082555
:10056600E0FF7403A807088002C333D8FCF53E55A4
:1005760013653E7053E53EF45213E4906100F0A318
:100586007408F0906402E0906102F0A374F0F0A3A6
:100596007402F0A37491F0E5082420A3F0E5083373
:1005A600333354F875F002A42403F582E5F034647D
:1005B600F58363A20190610763A2017F10122B45A8
:1005C6007F17123F230508220508020653E508C3D4
:1005D60094085076E50824FC25E0FF7403A8070874
:1005E6008002C333D8FCF53E5514653E7058E53E8F
:1005F600F45214E4906100F0A37408F0906402E0F1
:10060600906102F0A374F0F0A37402F0A37491F069
:10061600E50854032440A3F0E50833333354F87552
:10062600F002A42403F582E5F03464F58363A201A5
:1006360090610763A2017F10122B457F17123F239B
:1006460005085308072205088003E4F50890683872
:10065600E0701F906100F0A37408F0906402E090CF
:100666006102F0A37490F0E4A3F0A3F07F06123FBA
:100676002322906613E0FF7003020A19F53FE4F0A7
:10068600201D1F7E1C7F621233E2E53F5480243614
:10069600F582E43466AF82FEE53F547FFDE4FB124B
:1006A60035A5E53F7003020A19E53F5480FF24365D
:1006B600F582E43466AD82F5408D41E4F512F5111C
:1006C6008F3EE53EC3953F50180541E541AE40706B
:1006D60002054014F5828E83E0FF1241F7053E8045
:1006E600E1E51145126026301D03020A197E1C7FC2
:1006F6006A1233E2E53F54802436F582E43466AF6D
:1007060082FEE53F547FFDE4FB1235A522E49063AB
:1007160000F0A3F0D20D906184F0E53F54802436BA
:10072600F582E43466AF82F5408F4174022541F5C7
:1007360041E43540F540854182F583E0FF9064024F
:10074600E0FEEF6E6026301D03020A197E1C7F75DF
:100756001233E2E53F54802436F582E43466AF82F4
:10076600FEE53F547FFDE4FB1235A5220541E54138
:1007760070020540F582854083E0FFB43006E490C0
:100786006182F022EF64017003020A19EFB41805C2
:10079600D209D21022EFB4190B9062FEE0F513A332
:1007A600E0F51422854182854083E0FF54F064F031
:1007B60060030208A1906614EFF00541E54170025E
:1007C6000540F582854083E0FF648070330541E58E
:1007D6004170020540F582854083E0644060030273
:1007E6000A19D2120541E54170020540F58285409D
:1007F60083E064086003020A19D205906615F022A8
:10080600EFB401270541E54170020540F5828540B8
:1008160083E0644F6003020A19906839E0700302AE
:100826000A197408250EF50EE4F0228541828540EA
:1008360083E06003020A190541E54170020540F5AF
:1008460082854083E064426003020A190541E5415E
:1008560070020540F582854083E0906EE1F0054127
:10086600E54170020540F582854083E0906EE2F036
:100876000541E54170020540F582854083E0906EB2
:10088600E3F00541E54170020540F582854083E0CD
:10089600906EE4F0D224C205D212228541828540B0
:1008A60083E0FF64116008EF641260030209F7E554
:1008B6003F547F640E60030209F7201D077E1C7FEC
:1008C6007C1233E230220E301D03020A197E1C7F91
:1008D600911233E222854182854083E0540314F568
:1008E6003F0541E54170020540F582854083E0F50C
:1008F6003E30E709E4906EE0F0906EE5F0E53E30BC
:10090600E60BE4906EE0F0906EE57410F0E53E3094
:10091600E50B906EE07401F0E4906EE5F0E53E3094
:10092600E40C906EE07401F0906EE57410F0E53E14
:1009360030E30B906EE07402F0E4906EE5F0E53E75
:1009460030E20C906EE07402F0906EE57410F0E503
:100956003E30E10B906EE07403F0E4906EE5F0E556
:100966003E30E00C906EE07403F0906EE57410F08B
:1009760074022541F541E43540F540854182F58311
:10098600E0F53E30E700E53E30E607906EE5E02410
:1009960002F0E53E30E507906EE5E02404F0E53E22
:1009A60030E407906EE5E02406F0E53E30E307907C
:1009B6006EE5E02408F0E53E30E207906EE5E024BF
:1009C6000AF0E53E30E107906EE5E0240CF0E53EE6
:1009D60030E007906EE5E0240EF0906EE5E0253FEE
:1009E600F0D222E4906183F0906EDFF0906F67F0B2
:1009F60022201D1F7E1C7F9F1233E2E53F54802478
:100A060036F582E43466AF82FEE53F547FFDE4FBB3
:030A16001235A5F1
:010A190022BA
:1039EC00020A1AE493A3F8E493A34003F68001F2CD
:1039FC0008DFF48029E493A3F85407240CC8C333DC
:103A0C00C4540F4420C8834004F456800146F6DFAA
:103A1C00E4800B0102040810204080904236E47EC2
:103A2C00019360BCA3FF543F30E509541FFEE4939F
:103A3C00A360010ECF54C025E060A840B8E493A366
:103A4C00FAE493A3F8E493A3C8C582C8CAC583CA91
:103A5C00F0A3C8C582C8CAC583CADFE9DEE780BE49
:01423C000081
:101EF600BB010689828A83E0225002E722BBFE02EA
:091F0600E32289828A83E493221C
:101F0F00BB010CE58229F582E5833AF583E0225087
:101F1F0006E92582F8E622BBFE06E92582F8E222D1
:0D1F2F00E58229F582E5833AF583E49322EB
:101F3C00BC000BBE0029EF8DF084FFADF022E4CC89
:101F4C00F875F008EF2FFFEE33FEEC33FCEE9DEC52
:101F5C00984005FCEE9DFE0FD5F0E9E4CEFD22ED98
:101F6C00F8F5F0EE8420D21CFEADF075F008EF2FE2
:101F7C00FFED33FD4007985006D5F0F222C398FDD3
:051F8C000FD5F0EA2270
:101F9100A3F8E0C5F025F0F0E58215827002158303
:061FA100E0C838F0E82260
:101FA70075F008758200EF2FFFEE33FECD33CDCCF1
:101FB70033CCC58233C5829BED9AEC99E582984074
:101FC7000CF582EE9BFEED9AFDEC99FC0FD5F0D651
:101FD700E4CEFBE4CDFAE4CCF9A88222B800C1B97B
:101FE7000059BA002DEC8BF084CFCECDFCE5F0CBB9
:101FF700F97818EF2FFFEE33FEED33FDEC33FCEBF2
:1020070033FB10D703994004EB99FB0FD8E5E4F9AC
:10201700FA227818EF2FFFEE33FEED33FDEC33FC99
:10202700C933C910D7059BE99A4007EC9BFCE99A8D
:10203700F90FD8E0E4C9FAE4CCFB2275F010EF2FD2
:10204700FFEE33FEED33FDCC33CCC833C810D707D2
:102057009BEC9AE899400AED9BFDEC9AFCE899F80D
:0E2067000FD5F0DAE4CDFBE4CCFAE4C8F922A0
:0E207500C3E49FFFE49EFEE49DFDE49CFC227C
:10208300EB9FF5F0EA9E42F0E99D42F0EC6480C8D4
:0620930064809845F02274
:10209900EB9FF5F0EA9E42F0E99D42F0E89C45F09D
:0120A9002214
:0C20AA00ECF0A3EDF0A3EEF0A3EFF022A9
:1020B600A8828583F0D083D0821220CD1220CD1243
:1020C60020CD1220CDE473E493A3C583C5F0C58368
:1020D600C8C582C8F0A3C583C5F0C583C8C582C874
:0120E60022D7
:102C1C008B3D8A3E893FE4F549F548F547F546F585
:102C2C0044F545E541454245406012EBC0E0EAC041
:102C3C00E0E9C0E0AB40AA41A942122136AB3D0508
:102C4C003FE53FAA3E7002053E14F9121EF6F54A06
:102C5C00C394094007E54AD3940D40E1E54A64204A
:102C6C0060DBE54AB42D054345038016E54AB42BD9
:102C7C0005434501800C74FF253FF53F74FF353E3D
:102C8C00F53EE54360046410703FAB3DAA3EA93F9E
:102C9C00121EF664306009E543702E75430A8029D4
:102CAC00900001121F0FFF64786004EFB4581343B7
:102CBC0045017543107402253FF53FE4353EF53E62
:102CCC008007E5437003754308AB3D053FE53FAA1C
:102CDC003E7002053E14F9121EF6F54AC39461408B
:102CEC000AE54AD3947A5003534ADF74D0254AF547
:102CFC004AC3940A400CE54A9411406D74F9254A74
:102D0C00F54AE54AD39543506043450185494E85C4
:102D1C00484D85474C85464BAF437E00E4FCFDABEC
:102D2C0049AA48A947A8461220E7C8ECC8C9EDC96A
:102D3C00CAEECACBEFCBE4FCFDFEEB254AF549EE1F
:102D4C003AF548ED39F547EC38F546AF49AE48ADA4
:102D5C0047FCAB4EAA4DA94CA84BD312209950035B
:102D6C00022CD5434504022CD5E54520E003E48034
:102D7C002DE54145424540601EAB3DE53F24FFF942
:102D8C00E53E34FFFAEBC0E0EAC0E0E9C0E0AB405E
:102D9C00AA41A942122136E54530E20774FFFFFE35
:102DAC00FDFC22E545AF49AE48AD47AC4630E103EA
:042DBC00022075225A
:1020E700E88FF0A4CC8BF0A42CFCE98EF0A42CFC98
:1020F7008AF0EDA42CFCEA8EF0A4CDA8F08BF0A416
:102107002DCC3825F0FDE98FF0A42CCD35F0FCEB74
:102117008EF0A4FEA9F0EB8FF0A4CFC5F02ECD3939
:0F212700FEE43CFCEAA42DCE35F0FDE43CFC22A6
:10213600BB011A89828A83D0F0D0E0F8D0E0F9D0CA
:10214600E0FAD0E0FBE8C0E0C0F002218E5016E9CC
:10215600F8D083D082D0E0F9D0E0FAD0E0FBC0829C
:10216600C083022185BBFE16E9F8D083D082D0E079
:0F217600F9D0E0FAD0E0FBC082C08302219722AB
:09218500EBF608EAF608E9F6227F
:09218E00EBF0A3EAF0A3E9F02252
:09219700EBF208EAF208E9F22279
:00000001FF
